:020000040000FA
:100000000730990085018316850183121120A5010F
:10001000A7018030A30022202A203C20210885004F
:100020000B280330A000373085001B2085011B20E2
:10003000A00B13280800A401A601A60B1D28A40BE1
:100040001D2808000930A200851D2428A20A851950
:10005000262808002208230203183128A000A0093E
:10006000200AA00004302002031839282308A20027
:1000700008002208A300080050302202031842287A
:10008000A1010800A11421154C2080202110B030BE
:1000900022020318211408002508820759285D2828
:1000A00064286B28722879282112A40B0800A50166
:1000B00008000330A400A50A08002116A40B0800BC
:1000C0000830A400A50A08002112A40B0800033080
:1000D000A400A50A08002116A40B08000330A40000
:1000E000A50A08002112A40B08000330A400A50AE9
:1000F00008002116A40B08001E30A400A50A080061
:10010000270882078D28912898289F28A628AD289F
:10011000A112A60B0800A70108000330A600A70A39
:100120000800A116A60B08000830A600A70A0800C0
:10013000A112A60B08000330A600A70A0800A1160A
:10014000A60B08000330A600A70A0800A112A60B00
:1001500008000330A600A70A0800A116A60B080095
:080160001830A600A70A0800F0
:02400E0084012B
:00000001FF
